:0200000480007A
:1000000017110000130101001309000093080000FC
:10001000B338190323201101130A000093091000BB
:10002000B3393A0323223101130B0000930AF0FF86
:10003000B33A5B0323245101130C0000B70B00807B
:10004000938BFBFFB33B7C0323267101130D000050
:10005000B70C0080B33C9D032328910117110000C9
:10006000130181FB130E1000930D0000B33DBE037E
:100070002320B101130F1000930E1000B33EDF03D5
:100080002322D10193011000930FF0FFB3BFF103BE
:100090002324F10113041000370200801302F2FF41
:1000A000333244022326410093051000B704008038
:1000B000B3B495022328910017110000130101F732
:1000C0009306F0FF1306000033B6C6022320C100DA
:1000D0009307F0FF1307100033B7E7022322E10074
:1000E0009308F0FF1308F0FF33B80803232401013D
:1000F0009309F0FF370900801309F9FF33B9290389
:1001000023262101930AF0FF370A008033BA4A03FD
:100110002328410117110000130181F2B70B008061
:10012000938BFBFF130B000033BB6B032320610198
:10013000B70C0080938CFCFF130C100033BC8C03B5
:1001400023228101B70D0080938DFDFF130DF0FF79
:1001500033BDAD032324A101B70E0080938EFEFFB3
:10016000370E0080130EFEFF33BECE032326C101DF
:10017000B70F0080938FFFFF370F008033BFEF036F
:100180002328E101171100001301C1EC37020080A0
:1001900093010000B331320223203100B704008004
:1001A0001304100033B48402232281003706008038
:1001B0009305F0FFB335B6022324B1003707008062
:1001C000B70600809386F6FFB336D7022326D10008
:1001D00037080080B7070080B337F8022328F10002
:1001E00017150000130505E297150000938585EEAD
:1001F000370610F01306C6F26306B5028326C50063
:100200002320D600832685002320D60083264500A0
:100210002320D600832605002320D60013050501E0
:100220006FF09FFD370510F0130505F22320050040
:0402300000000000CA
:10100000FFFFFFFFFFFFFFFFFFFFFFFFFFFFFFFFF0
:10101000FFFFFFFFFFFFFFFFFFFFFFFFFFFFFFFFE0
:10102000FFFFFFFFFFFFFFFFFFFFFFFFFFFFFFFFD0
:10103000FFFFFFFFFFFFFFFFFFFFFFFFFFFFFFFFC0
:10104000FFFFFFFFFFFFFFFFFFFFFFFFFFFFFFFFB0
:10105000FFFFFFFFFFFFFFFFFFFFFFFFFFFFFFFFA0
:10106000FFFFFFFFFFFFFFFFFFFFFFFFFFFFFFFF90
:10107000FFFFFFFFFFFFFFFFFFFFFFFFFFFFFFFF80
:10108000FFFFFFFFFFFFFFFFFFFFFFFFFFFFFFFF70
:10109000FFFFFFFFFFFFFFFFFFFFFFFFFFFFFFFF60
:1010A000FFFFFFFFFFFFFFFFFFFFFFFFFFFFFFFF50
:1010B000FFFFFFFFFFFFFFFFFFFFFFFFFFFFFFFF40
:1010C000FFFFFFFFFFFFFFFF000000000000000028
:040000058000000077
:00000001FF
